:060000008831262F0000EC
:0800080083018A012000770842
:10001000A0007808A1007908A2007A08A3008B1E2E
:1000200013280B191C282008F7002108F8002208C3
:10003000F9002308FA0009008031E828F701F801E7
:100040002200240803102518F707F70CF80CA51850
:10005000F707F70CF80C2519F707F70CF80CA5199A
:10006000F707F70CF80C251AF707F70CF80CA51A88
:10007000F707F70CF80C251BF707F70CF80CA51B76
:10008000F707F70CF80C200008007930220023074E
:100090008400203085000318850A0008A400713010
:1000A00023078400203085000318850A0008A50076
:1000B0000310230D7D3E8400203085000318850A3F
:1000C000013FFA00003FA8007A08A9007530230715
:1000D0008400203085000318850A0008A6008530BA
:1000E00023078400203085000318850A0008A70034
:1000F000A208031D81282000AC01AB01AA01A901BF
:100100002200A40803198928A208031D89280130A8
:10011000A5002208A400A208031D99282808F43C81
:10012000031D9528290B95289928A80A0319A90ABF
:10013000AF28A208031DAF282808F43C031DAF28F0
:10014000290BAF280130A500A70A27080A3C03188D
:10015000AB280130A6000130A900C230A800A208D7
:100160000319B628A901A801A701A6017930230720
:100170008400203085000318850A2408800071302F
:1001800023078400203085000318850A2508800095
:100190000310230D7D3E8400203085000318850A5E
:1001A000280880002908813F75302307840020300B
:1001B00085000318850A26088000853023078400FF
:1001C000203085000318850A2708800020000800D9
:1001D00007309500270BA52A270BEF28F028A52A22
:1001E000720FFD28730FFD282200A2012208A10032
:1001F000F3017308F2002F29200073082200A400E5
:100200001430A50020001E2072087807153E8400D7
:10021000203085000318850A00082200A100F20A98
:100220007308A4001430A50020001E20720878076F
:10023000153E8400203085000318850A000822003E
:10024000A200F20A7208143C031D2F29F201F30ADE
:100250007308043C031D2F29FF30F300F2006430C3
:10026000A30021008C101F30F700F70B3529382927
:100270002200A11F3F2921008C14412922002100C6
:100280008C101F30F700F70B432946292200211F4D
:100290004D2921008C144F29220021008C101F3081
:1002A000F700F70B512954292200A11E5B292100D8
:1002B0008C145D29220021008C101F30F700F70BF1
:1002C0005F2962292200211E692921008C146B29D3
:1002D000220021008C101F30F700F70B6D297029C8
:1002E0002200A11D772921008C14792922002100E8
:1002F0008C101F30F700F70B7B297E292200211D6F
:10030000852921008C148729220021008C101F30A0
:10031000F700F70B89298C292200A11C93292100C1
:100320008C149529220021008C101F30F700F70B48
:1003300097299A292200211CA12921008C14A32984
:10034000220021008C101F30F700F70BA529A829E7
:100350008C141F30F700F70BAB29AE298C101F301F
:10036000F700F70BB129B4292200A21FBB292100F5
:100370008C14BD29220021008C101F30F700F70BD0
:10038000BF29C2292200221FC92921008C14CB2990
:10039000220021008C101F30F700F70BCD29D02947
:1003A0002200A21ED72921008C14D9292200210065
:1003B0008C101F30F700F70BDB29DE292200221EEC
:1003C000E52921008C14E729220021008C101F3020
:1003D000F700F70BE929EC292200A21DF3292100DF
:1003E0008C14F529220021008C101F30F700F70B28
:1003F000F729FA292200221D012A21008C14032A40
:10040000220021008C101F30F700F70B052A082A64
:100410002200A21C0F2A21008C14112A2200210084
:100420008C101F30F700F70B132A162A2200221C0B
:100430001D2A21008C141F2A220021008C101F303D
:10044000F700F70B212A242A8C140F30F700F70B42
:10045000272A2A2A20008C1C372A2200A308031DE1
:10046000332A2000372AA30321002A2A20001F3024
:10047000F700F70B392A3C2A0F30F700F70B3E2A1A
:10048000412A8C1C462A0130AD00472AAD011F309D
:10049000F700F70B492A4C2A8C1C512A0130AE0078
:1004A000522AAE011F30F700F70B542A572A8C1C32
:1004B0005C2A0130AF005D2AAF011F30F700F70B57
:1004C0005F2A622A8C1C672A0130B000682AB001BA
:1004D0001F30F700F70B6A2A6D2A8C1C722A013034
:1004E000B100732AB1011F30F700F70B752A782A83
:1004F0008C1C7D2A0130B2007E2AB2011F30F70029
:10050000F70B802A832A8C1C882A0130B300892AA1
:10051000B3011F30F700F70B8B2A8E2A8C1C932A0D
:100520000130B400942AB4011F30F700F70B962A6B
:10053000992A8C18A52A0130B000AF00AE00AD009A
:100540000130B400B300B200B1002D08F800780803
:100550002200A100A2000130A300200045202E08A7
:10056000F80078082200A100A200A3012000452085
:100570002F08F80078082200A100A2000330A30091
:10058000200045203008F80078082200A100A200D1
:100590000230A30020004520290FD62A2A0FD62A90
:1005A0002B0FD62A2C08073C0319DE2A0130A90795
:1005B0000318AA0A0319AB0A0319AC0A0B118031FC
:1005C00013282010CD2AD422201020002E186421B8
:1005D0002000AE1A64212000D020C722A5312000BF
:1005E00044284C263A00CC27C32500015527CC25AA
:1005F0000001A027D6212000201020102000AE1AD4
:10060000642100012E1864210000CD204927202BF1
:100610004F2620103A0041274126CF23202B4F267A
:100620003A00C1265010CD27C42220103A00E337EB
:10063000F232A0376E100001CC37772369102010FA
:100640000001C834C634A01856100001C834C6349E
:1006500020195610000048282010C224C12920105B
:100660003A00C8244724201020100001CC2757103E
:10067000201020100001C6244C2A452920102010EB
:100680003A0044284C26A02766330000CC27C32517
:10069000A029D02245223A00C22BA024B2292F2221
:1006A0006F283A00C22B20225322201020103A003B
:1006B000C4375010CC37E73463103A004537613106
:1006C000EC3220100001C434F330623665100001B2
:1006D000C23CF030F339202A48223A00C434F330C7
:1006E00062366510000145376131EC32201000019F
:1006F0004927492AC920CC24DA223A284129C115A0
:10070000C72721004927D42252274126A022522957
:100710004F290000D034C420C31CB218381053260F
:10072000412B4510CD27C4220001202B65393117FC
:10073000301032183218AD26E13C2D193710000167
:100740002014E314CF254929C1255510C12AC424FA
:100750004F10201000008501EF30840000080319BD
:10076000BE2B0A30F800F701F70BB42BF80BB32BB4
:100770005F30F700F70BBA2B800BB12B080021007C
:10078000D9080319CA2B0A30EF002000AB2321003F
:10079000D903C02B20000800FF3021008C008D0001
:1007A00024008D00210095138C1122008D1621004C
:1007B0008D120D1622000C1321000C13883120001D
:1007C000732F270B192C2100D9015908033C031C56
:1007D0000C2CDA015A08133C031C0A2C2000A4013B
:1007E0008B1BA4178B13210059082200A40014307E
:1007F000A50020001E20A41B8B1721005A08780793
:10080000153E8400203085000318850A20308000C2
:10081000DA0AEA2BD90AE52B22008C1021008C146D
:10082000F001F101FF30F300F2006430EF0020002E
:10083000AB2388317F2F270B4F2C2100D90159087A
:10084000033C031C462CDA015A08133C031C442CBD
:100850002000A4018B1BA4178B1321005908220030
:10086000A4001430A50020001E20A41B8B1721001B
:100870005A087807153E8400203085000318850A41
:1008800020308000DA0A242CD90A1F2CF001F10153
:10089000FF30F300F2000230EF002000AB2388317C
:1008A000822F270B7B2CA4018B1BA4178B137108A1
:1008B0002200A4001430A50020001E20A41B8B17CA
:1008C00070087807153E8400203085000318850ADB
:1008D000210067088000F00A7008143C031D762C84
:1008E000F001F10A7108043C0319F1016A30F700C4
:1008F000F70B782C00002000080023009517151432
:100900000000000013087F390319BF2C2100E40008
:10091000230011082100E500230012082100E60051
:100920006408E7002000512421006508230091009D
:10093000210066082300920095171514000000009E
:10094000130D140D7F390319BF2C2100E40023007F
:1009500011082100E500230012082100E6006408C8
:10096000E7002000512421006508230091002100A8
:10097000660823009200910A0319920A7E2C200037
:10098000080021006408230091002100650823006D
:100990009300951315150B08F7008B13553096002F
:1009A000AA30960095149518D32C151177088B044E
:1009B0002000080022008D160530F700F70BDE2C12
:1009C0000D1221000D120530F700F70BE52C220067
:1009D0008D120530F700F70BEB2C200008002100EA
:1009E0000D160530F700F70BF32C22008D1605309D
:1009F000F700F70BF92C8D120530F700F70BFE2CE2
:100A00002000080022000D1221000D120530F70011
:100A1000F70B082D22008D160530F700F70B0E2D71
:100A20008D120530F700F70B132D20000800210070
:100A3000EE016E08063C031C2A2DED1F232D20001D
:100A4000EF24252D21002000022503102100ED0DAB
:100A5000EE0A192D200008002100ED010D160530C9
:100A6000F700F70B312D22008D160530F700F70B3C
:100A7000372D20000D1E4C2D0530F700F70B3E2DB5
:100A80002100ED0A6D08643C031D492D20004C2D0A
:100A900021002200392D200022008D120530F700A0
:100AA000F70B502D0530F700F70B542D0D122100D8
:100AB0000D120530F700F70B5B2D6D08643C031D2C
:100AC0007B2DEE016E08093C031C772D22008C154E
:100AD00032302100EF002000AB2322008C11643063
:100AE0002100EF002000AB232100EE0A622D01302F
:100AF000F8007E2D7E2D0030F8007E2D20000800AD
:100B000022000D1221000D120530F700F70B862D83
:100B100022008D160530F700F70B8C2D21000D16E5
:100B20000530F700F70B922D2000080090302100CF
:100B3000E9006608EA006708EB0069082000A500E4
:100B4000DA2421006908ED002000172502252C2554
:100B5000F8080319AF2D80250130F800EA2D210097
:100B6000EC016C08073C031CC22DEA1FBB2D2000C2
:100B7000EF24BD2D21002000022503102100EA0DE5
:100B8000EC0AB12D20002C25F8080319CB2D802567
:100B90000130F800EA2D2100EC016C08073C031C31
:100BA000DE2DEB1FD72D2000EF24D92D21002000B2
:100BB000022503102100EB0DEC0ACD2D20002C2581
:100BC000F8080319E72D80250130F800EA2D80256B
:100BD0000030F80078082100E8002000080021001B
:100BE0006308013A20000319202E023A0319282E27
:100BF000053A0319342E013A0319472E0F3A031907
:100C0000552E023A03195D2E063A0319652E013A54
:100C10000319742E023A0319862E143A03199B2ED7
:100C20003B3A0319A32E0D3A0319B42E033A0319C4
:100C3000BC2E013A0319C32E1F3A0319CB2EDE2E08
:100C400001302100E6008E30E70020009625DF2EDF
:100C50007408183C40382100E5000330E6006508C0
:100C6000E70020009625DF2EF50803193F2E0630F9
:100C70002100E6007A30E70020009625462E063057
:100C80002100E6007230E70020009625DF2E760E68
:100C90002100E400E40DE030E405E4050730E6005F
:100CA0006408E70020009625DF2E08302100E600CA
:100CB000BB30E70020009625DF2E0A302100E60039
:100CC0007B08E70020009625DF2E7C0E2100E40043
:100CD000F030E405E4057D08E4040C30E600640827
:100CE000E70020009625DF2EFE0803197F2E0D3029
:100CF0002100E6004030E70020009625852E0D30CB
:100D00002100E600E70120009625DF2E21003508AE
:100D1000FF3CE5000F30E6006508E700200096255F
:100D200021003508FF3CE5001030E6006508E700CB
:100D300020009625DF2E1B302100E600DC30E70086
:100D400020009625DF2E2100360DF700F70DF70D58
:100D5000F830F70577083604E5002030E60065082E
:100D6000E70020009625DF2E2D302100E6007C30A4
:100D7000E70020009625DF2E2E302100E600E70157
:100D800020009625DF2E2F302100E6007F30E7007F
:100D900020009625DF2E2100B7080319D72E30300A
:100DA000E6004830E70020009625DD2E2100303097
:100DB000E6004030E70020009625DF2EDF2E0800F9
:100DC000270BFA2E21005F08F0006008F100643064
:100DD000E2000230E202031CFA2E2030850092303D
:100DE000840000080319FA2EF82EF62EF72E0000C4
:100DF000800BF52E2000080021005E082000A500D1
:100E0000DA2421005E08ED002000172502252C259C
:100E1000F80803190F2F80250130F800912F2100C9
:100E2000E0016008073C031C222FDF1F1B2F20005E
:100E3000EF241D2F21002000022503102100DF0DCB
:100E4000E00A112F22008D160530F700F70B262F30
:100E500021000D160530F700F70B2C2F22008D1204
:100E60000530F700F70B322F8D160530F700F70B22
:100E7000372F0D1221000D120530F700F70B3E2F12
:100E800022008D120530F700F70B442F21005E0879
:100E9000ED0020001725EF242C25F8080319542F06
:100EA00080250130F800912F2100E101E001600868
:100EB000073C031C7C2F0310E10D0D1622008D163C
:100EC0000530F700F70B622F20000D1E6C2F01304C
:100ED0002100E2006E2F20002100E20122008D128D
:100EE0000530F700F70B722F21006208F800F808B0
:100EF000031D6114E00A572F0D160530F700F70B9C
:100F00007F2F22008D160530F700F70B852F8D12ED
:100F10000530F700F70B8A2F20008025210061089B
:100F2000F8002000080021006508F8016402031899
:100F30009C2F6408F700A82FF7010830E600E40DA5
:100F4000F70D650877020318F700F80DE60B9F2FE1
:100F5000200008002100DE080319B42F3E30E7000E
:100F600020005124B82F21002030E7002000512418
:100F7000080021005E08E4000A30E5002000932705
:100F8000303078072100E1005E08E4000A30E50017
:100F900020009327303077072100E2002330E7005C
:100FA0002000512421006108E70020005124210085
:100FB0006208E700200051242100E0015F08600280
:100FC0000318E92F2030E700200051242100E00A17
:060FD000DE2F20000800E6
:101000002100DF01E00180312000E026883130300E
:1010100021005D07DE00EC302300910002309200D9
:10102000031004302100DF00230095171514000081
:1010300000000318412813087F392100E000230035
:1010400011082100E100230012082100E2006008DD
:10105000E7008031200051248831210061082300FD
:1010600091002100620823009200951715140000DA
:1010700000002100DF0B3D283F2823004128632882
:101080002300130D140D7F392100E0002300110807
:101090002100E100230012082100E2006008E700BF
:1010A0008031200051248831210061082300910003
:1010B0002100620823009200910A0319920A03108A
:1010C0002100DF0B14285E08E70080312000512446
:1010D000883120302100E700803120005124883100
:1010E000F0302300910002309200803120007D24F6
:1010F000883190302100DE004030DF008031200058
:10110000FC268831781C8E28F330230091000230B1
:101110009200803120007D2488319728F63023000A
:10112000910002309200803120007D24883190307F
:101130002100DE004830DF0080312000FC268831AD
:101140007808C0390319AE28F93023009100023025
:101150009200803120007D248831B728FC302300A4
:10116000910002309200803120007D2488310800F7
:10117000031021005D0CDE005E08633C0318DF28CD
:101180002D30DF003130E0006430DE025E08E40024
:101190000A30E50080312000932788317808303EFE
:1011A0002100E1005E08E4000A30E5008031200003
:1011B000932788317708303E2100E20008295E0835
:1011C000093C031800292030DF002D30E0005E08C4
:1011D000E4000A30E5008031200093278831780848
:1011E000303E2100E1005E08E4000A30E500803175
:1011F0002000932788317708303E2100E20008293B
:101200002030E000DF002D30E10030305E07E200EA
:10121000E301203085008F308400800803192329E2
:101220000508E5000408E4000008E700803120001C
:101230005124883121006508850064088400840AEF
:101240000319850A0D295D1C3029FF302300910008
:1012500002309200803120007D248831392921001C
:1012600002302300910003309200803120007D2461
:101270008831080001302100DD002000002001300D
:101280002100DF00E00080312000E02688310530B9
:101290002300910003309200803120007D248831AA
:1012A00021003508FF3CDC00DD002000B8200130C3
:1012B0002100DF000230E00080312000E02688318C
:1012C0000B302300910003309200803120007D24F8
:1012D00088310310740D303C2100DC00DD0020005B
:1012E000B82001302100DF000330E0008031200011
:1012F000E0268831113023009100033092008031C4
:1013000020007D24883121003608003A200003198E
:101310009329013A03199D29033A0319A729013A90
:101320000319B129BB291730230091000330920023
:10133000803120007D248831BC291C30230091009D
:1013400003309200803120007D248831BC29213077
:101350002300910003309200803120007D248831E9
:10136000BC292630230091000330920080312000F8
:101370007D248831BC29BC292100DF010130E00037
:1013800080312000E02688312100DB080319CA29BA
:101390000030CB290130DC00DE0080312000AA279C
:1013A00088312100DF010230E00080312000E0269A
:1013B000883121005B0BDD29DF290030E029013075
:1013C000DC00DE0080312000AA2788312100DF0107
:1013D0000330E00080312000E026883121005B08E6
:1013E000023C0319F5290030F6290130DC00DE004B
:1013F00080312000AA278831080021006208023CC1
:10140000031D2A2A5D08FA005C0884005D08850037
:101410005F0800020319112A5C0884005D0885003A
:10142000800A5D08FA005C0884005D0885000008F9
:10143000E3006008E4006308E50080312000C12477
:10144000883121005B08E30080312000EF258831DE
:10145000542A21006208033C031D552A5D08FA0046
:101460005C0884005D0885005E08000203193D2ABF
:101470005C0884005D08850080035D08FA005C0854
:1014800084005D0885000008E3006008E40063084C
:10149000E50080312000C124883121005B08E30091
:1014A00080312000EF258831210020000800210034
:1014B0006108023C031D8C2A5D08FA005C08840068
:1014C0005D0885005E080002031D6E2A5D08FA00B3
:1014D0005C0884005D0885008001732A5C08840034
:1014E0005D088500800A5D08FA005C0884005D08DC
:1014F00085000008E2005F08E4006208E500803132
:101500002000C124883121005B08E30080312000E5
:10151000EF258831BE2A21006108033C031DBF2A44
:101520005D08FA005C0884005D0885008008031DE2
:10153000A22A5D08FA005C0884005D0885005E0848
:101540008000A72A5C0884005D08850080035D0890
:10155000FA005C0884005D0885000008E2005F086E
:10156000E4006208E50080312000C12488312100B8
:101570005B08E30080312000EF2588312100200046
:10158000080002302100DD00200000200130210091
:10159000DF00E00080312000E02688312B3023007E
:1015A000910003309200803120007D248831210099
:1015B000B7080319E62A3130230091000330920066
:1015C000803120007D248831EF2A2100363023002D
:1015D000910003309200803120007D248831013059
:1015E0002100DF000230E00080312000E026883159
:1015F0003B302300910003309200803120007D2495
:10160000883176082100DE000630DF0080312000BE
:10161000B927883103302100DD00DF015D08E000DB
:1016200080312000E02688312100DE015E08133C75
:10163000031C232B2030E700803120005124883107
:101640002100DE0A162BDF010130E000803120008E
:10165000E02688312100DC080319302B0030312BC3
:101660000130DD00DE0080312000AA278831210012
:10167000DF010230E00080312000E02688312100C7
:101680005C0B432B452B0030462B0130DD00DE0088
:1016900080312000AA27883108002100DD08031DC1
:1016A0005C2B4130230091000330920080312000F8
:1016B0007D248831642B21005D08DE000530DF00C9
:1016C00080312000B9278831080003302100DD0077
:1016D0002000002001302100DF00E00080312000E8
:1016E000E02688314630230091000330920080319B
:1016F00020007D2488317B082100DE000530DF00DA
:1017000080312000B927883101302100DF0002300C
:10171000E00080312000E02688314C302300910029
:1017200003309200803120007D2488317C08210024
:10173000DD0020004D2301302100DF000330E000F8
:1017400080312000E02688315230230091000330A0
:101750009200803120007D2488317D082100DD0049
:1017600020004D232100DF010130E0008031200006
:10177000E02688312100DC080319C02B0030C12B82
:101780000130DD00DE0080312000AA2788312100F1
:10179000DF010230E00080312000E02688312100A6
:1017A0005C0BD32BD52B0030D62B0130DD00DE00B7
:1017B00080312000AA2788312100DF010330E000BA
:1017C00080312000E026883121005C08023C0319AA
:1017D000EB2B0030EC2B0130DD00DE0080312000EF
:1017E000AA278831080004302100DD0020000020F5
:1017F00001302100DF00E00080312000E026883148
:1018000058302300910003309200803120007D2465
:101810008831F5080319162C5E302300910003303F
:101820009200803120007D2488311F2C63302300FA
:10183000910003309200803120007D2488310130F6
:101840002100DF000230E00080312000E0268831F6
:1018500068302300910003309200803120007D2405
:101860008831FE0803193E2C6E30230091000330AE
:101870009200803120007D248831472C7330230072
:10188000910003309200803120007D2488310130A6
:101890002100DF000330E00080312000E0268831A5
:1018A00078302300910003309200803120007D24A5
:1018B00088312100DF010130E00080312000E02686
:1018C00088312100DC080319672C0030682C0130B6
:1018D000DD00DE0080312000AA2788312100DF01F1
:1018E0000230E00080312000E026883121005C0BCE
:1018F0007A2C7C2C00307D2C0130DD00DE00803124
:101900002000AA2788312100DF010330E000803168
:101910002000E026883121005C08023C0319922C4B
:101920000030932C0130DD00DE0080312000AA273A
:10193000883108002100DB01DC015C08063C031C47
:10194000B62C5C0823009100951315141308210090
:10195000DD0069305C078400203085000318850AAB
:1019600000085D02031DDB0ADC0A9D2C5B08F80001
:10197000F80803194A2DDC015C08063C031CD42C32
:1019800069305C078400203085000318850A000850
:10199000DD005C08E4005D08E50080312000C12422
:1019A00088312100DC0ABC2C1830F4000A30E40035
:1019B0007408E50080312000C1248831F5010B3026
:1019C0002100E4007508E50080312000C124883141
:1019D0000430F6000C302100E4007608E500803188
:1019E0002000C12488310230FB000D302100E400CA
:1019F0007B08E50080312000C12488310530FC00DF
:101A00000E302100E4007C08E50080312000C12474
:101A100088310A30FD000F302100E4007D08E50028
:101A200080312000C12488310130FE0010302100B7
:101A3000E4007E08E50080312000C1248831FF30B9
:101A40002100B5001130E4003508E50080312000A8
:101A5000C124883103302100B6001230E40036087A
:101A6000E50080312000C12488312100B701133006
:101A7000E4003708E50080312000C12488312100CE
:101A8000B8011430E4003808E50080312000C1249A
:101A9000883121000A302300910095131514130892
:101AA000F4000B309100951315141308F5000C3059
:101AB0009100951315141308F6000D30910095133D
:101AC00015141308FB000E3091009513151413081C
:101AD000FC000F309100951315141308FD00103011
:101AE0009100951315141308FE0011309100951301
:101AF000151413082100B50012302300910095132E
:101B0000151413082100B60013302300910095131B
:101B1000151413082100B700143023009100951309
:101B2000151413082100B8000130DA005A08303CBF
:101B3000031CA32D5A08E30080312000EF258831D3
:101B40002100DA0A962D0A302000A6002100C208E2
:101B50000319AE2DC2010130F800C52DC1080319CB
:101B6000B52DC1010030F800C52DC4080319BC2DE6
:101B7000C4010330F800C52DC3080319C32DC301E8
:101B80000230F800C52DFF30F8007808D900380879
:101B9000003A20000319EB2D013A0319022E033AF3
:101BA0000319182E013A03192D2E073A0319452E51
:101BB000013A03195C2E033A0319742E013A0319F2
:101BC0008C2E0F3A0319A32E013A0319BA2E033AA9
:101BD0000319D12EE82E21003808DB0020003A211D
:101BE0000F302100DB002030DD006530DC00DE013D
:101BF000FF30DF00E1011130E0005908E200200071
:101C0000FD21F22E21003808DB0020003A210330AC
:101C10002100DB00DD017430DC00DE011830DF0064
:101C2000E1010A30E0005908E2002000FD21F22E17
:101C300021003808DB0020003A2120302100DB00A1
:101C4000DD006630DC000330DE00E0011230DF0032
:101C50005908E10020005722F22E033021003802FB
:101C6000DB00DC002000C12230302100DB0020300E
:101C7000DD006730DC000130DE00E0011330DF0002
:101C80005908E10020005722F22E033021003802CB
:101C9000DB00DC002000C12207302100DB00DD0179
:101CA0007630DC000730DE00E0010C30DF00590840
:101CB000E10020005722F22E053021003802DB001F
:101CC000DC00200065230A302100DB00DD017B30D1
:101CD000DC00DE010F30DF00E1010D30E0005908CB
:101CE000E2002000FD21F22E053021003802DB0049
:101CF000DC00200065230C302100DB00DD017C309E
:101D0000DC00DE010F30DF00E1010E30E000590899
:101D1000E2002000FD21F22E053021003802DB0018
:101D2000DC00200065230C302100DB00DD017D306C
:101D3000DC00DE010F30DF00E101E0005908E200C5
:101D40002000FD21F22E083021003802DB00DC00EB
:101D50002000F32306302100DB00DD017530DC00BC
:101D60000130DE00E0010B30DF005908E100200007
:101D70005722F22E083021003802DB00DC00200060
:101D8000F3230D302100DB00DD017E30DC0001306B
:101D9000DE00E0011030DF005908E100200057228A
:101DA000F22E083021003802DB00DC002000F32393
:101DB00021005908023C031DE62EE4012A30E5000B
:101DC00080312000C1248831010021002000F22E42
:101DD00082302300910003309200803120007D2466
:101DE0008831F22E21005908DB005B08003A200000
:101DF0000319FE2E013A03190F2F222F2608210066
:101E000038020319052FB80A062FB8011430E40070
:101E10003808E50080312000C1248831232F2100BB
:101E2000B808031D182F200026082100B800192F1C
:101E3000B8031430E4003808E50080312000C124E4
:101E40008831232F232FA62D8831D62F8501840199
:101E50001F308305F4302100990001302000A700D5
:101E6000A800AD00AE00AF00B000B100B200B300FA
:101E7000B40023008C018D01220092019101940194
:101E800093014F302100B9004B30BA004930BB00FC
:101E90005230BC004130BD004B30BE005530BF0059
:101EA000C001C101C201C301C401C501C601C7010E
:101EB000C801C901CA01CB01CC01CD01CE01CF01BE
:101EC000D001D101D201D301D401D501D601D7016E
:101ED000D801F0309900F430D90080312000BF23C0
:101EE00088318031CC2B883114302100D9008031E9
:101EF0002000BF2388310130A7008031E12B8831D9
:101F000080311B2C883122000C130230F700F70BB4
:101F1000872F00000C170A302100EF0080312000CD
:101F2000AB23883121001508C039043895000730EB
:101F3000200095008B16C0308B048A30230091005E
:101F400003309200803120007D24883195302300B9
:101F5000910003309200803120007D248831A03030
:101F60002300910003309200803120007D248831CD
:101F700022008C1502302100D900FA30EF008031A8
:101F80002000AB2388312100D90BBD2F22008C11FA
:101F900006302100D900FA30EF0080312000AB2359
:0E1FA00088312100D90BCB2F20009A2C630032
:020000040001F9
:04000E000439FF1E94
:00000001FF
